:10000000CB28A4008417800484138E010C1C8E005E
:1000100023200319C62823200319C6282320C62815
:10002000A40059200C080D040319C628C02084130D
:100030002408800664001C281D288C0A03198D0FD3
:100040001A288006C62824088E0601308C008D01EF
:10005000000824050E06031D08008C0A03198D0FE5
:10006000282808008F002608840024095A208413B9
:100070008F080319C628F03091000E0880389000D0
:10008000F03091030319910003198F030319C62857
:1000900049285D2003010C1824088E1F24088E08AF
:1000A00003190301900F562880063D2857280000A9
:1000B0004028FF3A84178005C6280D080C04031950
:1000C0008C0A80300C1A8D060C198D068C188D0642
:1000D0000D0D8C0D8D0DC6288F018E00FF308E0703
:1000E000031C8F07031CC62803308D00DF307A20E5
:1000F0006E288D01E83E8C008D09FC30031C83289E
:100100008C07031880288C0764008D0F80280C183A
:1001100089288C1C8D2800008D2808008E00033053
:1001200094288E000430942894000F080D02031DBB
:100130009B280E080C02043003180130031902300A
:100140001405031DFF30C628910190011030920064
:100150000D0D900D910D0E0890020F08031C0F0F4E
:1001600091020318BA280E0890070F0803180F0F02
:10017000910703108C0D8D0D920BA8280C08C62832
:100180008C098D098C0A03198D0A08008313031347
:1001900083126400080083168501083086008312EC
:1001A0000611831606118312861083168610831299
:1001B00006108316061083120130CB00640006304F
:1001C0004B020318E6288B21CB0FDE28BE01BF01AE
:1001D000C50164000B3045020318FB28D52103102C
:1001E000450D283E840040088000840A41088000B4
:1001F000B021C50FE9280B30C400C50164000B30E5
:100200004502031823290310450D283E84000008E9
:100210009E00840A00089F000310440D283E8400BD
:100220000008A000840A0008A1001E088C001F0816
:100230008D0021088F0020089120031D21294508E9
:10024000C400C50FFE2844080B3CC8000130CB0099
:1002500064004B084802031C30298B21CB0F28294E
:100260000130CB00640010304B0203184629D52121
:1002700040088C0041088D008F0106308E20031D40
:1002800043295A21DC284921CB0F3229DC2863007D
:100290004729AA30C700F421A030C600A030C90009
:1002A000F4216430C700F4217830C6007830C900EA
:1002B000F4210800CB01640004304B0203188A29A2
:1002C0000630A6001030A4005A308E0001303220D3
:1002D00050308E00023032207D308E0001303220CE
:1002E0005A308E000230322064308E0002303220CC
:1002F000AA30C700F4217830C6007830C900F42154
:100300006430C700F421A030C600A030C900F42139
:10031000CB0F5B2908000630A6001030A4008C30FB
:100320008E000130322050308E00023032207D307D
:100330008E00013032205F308E0002303220AA3031
:10034000C700F4217830C600A030C900F421643021
:10035000C700F421A030C6007830C900F42108009D
:100360000630A6001030A4008C308E000130322000
:1003700078308E00023032206E308E000130322014
:1003800064308E0002303220AA30C700F421A03041
:10039000C6007830C900F4216430C700F4217830F9
:1003A000C600A030C900F421080001308C008D0186
:1003B000063084000430102001308C0006308400A8
:1003C000083001200C08C2000D08C30042088C0050
:1003D00043088D000F308E008F01A420C0000D084F
:1003E000C10001306C2008000130CA0064000B30ED
:1003F0004A020318142A47088C008D010630840035
:100400008030102046088C008D010630840040307A
:10041000102049088C008D01063084002030102007
:0A0420000D306C20CA0FF629080009
:02400E00F53F7C
:00000001FF
